:020000040000FA
:020000002528B1
:08000800832AB80000308A00D1
:10001000383038028207F8344734F834F434F9348D
:100020005934F934B934FA341334FA346834FA34BC
:10003000B934FB340434FB344C34FB349034FB349B
:10004000CF34FC340C34FC34443483018B0103136F
:1000500083128501870107309900831691010E30C4
:10006000850000308700083081000C1083128B124D
:1000700001309000870185010B178B177F2205083F
:100080000639063A03193F28792205080639063A47
:10009000031D4528792249225B20812283162630C0
:1000A0009B001C141A088312A600A700A401A50136
:1000B00027089F20BF2861208020612080206120A8
:1000C00008000730AC000130AB00AC030319702806
:1000D0002B088700752287017B220310AB0D652852
:1000E0000330AC001030AB00AC0303197F282B08A1
:1000F0008500752285017B220310AB0D7428080052
:100100000230AC001030AB00AC0303198F282B0871
:100110008500752285017B220310AB0C84280630F4
:10012000AC002030AB00AC0303199E282B088700DD
:10013000752287017B220310AB0C932808008701EE
:100140008501AA20AB003F398700AB0C2B0C30395E
:1001500085000800B80000308A00380882070034A3
:1001600001340234043408341034203440348034F0
:1001700081348234843488349034A034C0340519F6
:10018000DB288B1224107722DC30AC00013068228F
:100190000519D228AC0BC628A703270A0F3003196C
:1001A000A700D728A70A2708103C0319A70127088A
:1001B0009F208122BF28851C22292418E7288B1222
:1001C00024140130A8001E30A900C821BF28280827
:1001D000031DBF288B122410870185012708031DEA
:1001E000F3282608A7000130A8000630A900C8217E
:1001F000A501280803190F2925184D22A501050876
:100200000639063A0319F9288B12792205080639AE
:10021000063A031D0629792227089F20BF288B1242
:10022000A5015B22542287018501831606309600C2
:1002300083128B15630005080639063A0319152940
:10024000792206298B12270803198529A8003C303A
:10025000A900C821870185012514251C43292808E8
:100260009F20752287018501A50129083C3C0319BF
:100270004522280B432929080A3C03183722290B59
:1002800043298022462985182D29A4018B12870134
:10029000850124184E295B227F228129A401270889
:1002A000260203196429831626309B00831227082F
:1002B000A60083169A001C1555309D00AA309D009B
:1002C0009C149C1861298312851973290530AC0090
:1002D0004922851C812977224922851C8129812276
:1002E000AC0B682981290230AC00851C81290230C1
:1002F000B3001A30B400D021851C81297F22AC0BB9
:10030000752927089F208022BF28A401A901A801E0
:10031000AA01C8212514251CBA29A5012903031DFA
:100320009D292A08B800B8080319BA2937227D2266
:100330007D22B8032518A501932929080319A829A6
:10034000B8000530B8020319A8290318A129BA2951
:100350002808031DB029372229080319B829BA290A
:100360009F207522870185012908031DBA2937229C
:100370007522452208302A020319C02985188B29C5
:100380008B1280225B222608A7009F208022BF2894
:10039000383081001230A0002730A1008B160800F1
:1003A0000130B2001122AF002F080319082A1122D0
:1003B000B00080302F020319FA29C0302F02031D2C
:1003C000E4293008B100052AC1302F02031DEF29AE
:1003D0003308B5003408B6003008B200052A03100F
:1003E0002F0D0520A20003142F0D0520A300831656
:1003F0000C1483123108B70001306822B70BFC29B6
:10040000B00BFA2983160C1083128518D229102AF2
:10041000B20B0B2A102A3508B3003608B400D229D3
:1004200008001622B40A0319B30A080033088A0028
:1004300034088200C0342334803408342334043434
:100440002534043427341834253404342334043454
:1004500080340C34233404342534043427340434F5
:100460002534043423340434253420340034FB3060
:10047000A2000430A300643060220800FC30A20017
:100480004430A300643060220800372275223722EE
:100490000800372277223E220800F830A200893077
:1004A000A300643060220800F830A2008930A30065
:1004B000FA30602208004D2264306822542208007D
:1004C00083160C148312682283160C108312080002
:1004D000AD006E30AE006C2A6D2A6E2AAE0B6B2A10
:1004E000712A722AAD0B692A08000F30682A1E3063
:1004F000682A3230682A5530682A6430682A802297
:100500008122FA30682AF0000308F10083120B19E7
:100510008E2A0C18BB2A0B18C32AC82A0B11383094
:1005200081000130A1020319992A0318C82AA002E8
:10053000C82AA008031DC82A1230A0002730A10035
:10054000251427080319AA2AA90BC82A3C30A90098
:10055000A803C82A2418A42AA90A3C302902031D8A
:10056000C82AA901A80A10302802031DC82A013090
:10057000A800AA0AC82A0C1022088F0023088E009F
:1005800001308506C82A0B108B1183169601831241
:0A05900071088300F00E700E0900E0
:02400E00C43CB0
:1042000043006F0070007900720069006700680069
:1042100074002000280043002900200032003000F4
:10422000310039002D003200300032003000200013
:104230006200790020004D002E00590061006D00E1
:0E42400061006D006F0074006F00FF0003004E
:00000001FF
